:10000000370101007128A948730000008280148123
:10001000988133E6E60009C685050505E389E6FE15
:1000200013351600828052B82A84D12C2A94C12C10
:10003000E36F85FE52BE8AB84D2C25C113044006DD
:1000400093045006130940079309300619A0712C38
:1000500029C50145C1240808C1450A86C146592C55
:1000600003450101E31585FE03451101E31195FEEA
:1000700003452101E31D25FD03453101E31995FCED
:1000800003454101E31535FD03455101E31125FD0C
:10009000034561014DFD05458ABE0545A52C8ABC79
:1000A000FAB8130560352D241305C0361524130442
:1000B000E0389305403922852524130580399305BE
:1000C000D039392C1305103A9305603A112C130BD3
:1000D000903A930BC0417EAF2124052C9304400637
:1000E00093095006930A400713093006130C804504
:1000F000930C4046130D70461305003BD12A05456D
:10010000112C1305603BE922CD2221C5014519249C
:100110000808C1450A86C146F12A03450101E315D5
:1001200095FE03451101E31135FF03452101E31D50
:1001300055FD03453101E31935FD03454101E31543
:1001400025FD03455101E31155FD034561014DFDB9
:1001500021A00545C1224DBF1305703C952A0145DC
:10016000552A130580399305803E9D2A1305B03E1C
:10017000852222859305503FA5221305C03F892A79
:10018000BD2A130A3500A52AE36F45FF7EAC892AF4
:100190001305B040352AA522130A15008D22E36FFE
:1001A00045FF228593057041252A130500420D2243
:1001B000B922130A5500A122E36F45FF1305103A37
:1001C00093052043312A1305704319220D2A130A7F
:1001D00045003522E36F45FF5A85930530440922D7
:1001E00013059044F52015223D4A09A805451D2216
:1001F00001450D227D1A1375FA0F3DC9937DFA0F43
:100200006285F9206E85C9206685D920CD28930D99
:100210001500F520E36FB5FFC92869D90145DD2830
:100220000808C1450A86C146F12003450101E315CE
:1002300095FE03451101E31135FF03452101E31D3F
:1002400055FD03453101E31935FD03454101E31532
:1002500025FD03455101E31155FD034561014DFDA8
:10026000552865206A85AD20614A1375FA0F59F546
:100270001305C047B1287EAFA52013057048892813
:10028000130580399305D039A128130540498920E9
:10029000BD20130A1500A520E36F45FF1305103A92
:1002A0009305603A35281305F0491D208928130A63
:1002B0002500B120E36F45FF2285930540390D20CD
:1002C0001305904A31200DBD8548730000008280DF
:1002D0009148730000008280AD4873000000828066
:1002E0009308100873000000828093085008730080
:1002F00000008280930870087300000082807325DC
:1003000010C08280732500C082809308600873004B
:10031000000082800589F322008093920248B3E2B4
:10032000A200739002808280954873000000828052
:1003300093080008730000008280A1487300000049
:100340008280930830087300000082809308400880
:10035000730000008280554B205261696C726F619E
:10036000642043726F7373696E670A00666F722050
:100370005256436F6E74726F6C6C65720A496E6987
:100380007469616C697A696E672048570A006C6904
:10039000676874004F46460062656C6C006F666665
:1003A0000067617465007570007369676E616C0049
:1003B00049646C650A004C696768747765696768A9
:1003C000743A204F6E0A00547261696E206465743D
:1003D00065637465640A4C69676874776569676802
:1003E000743A204F66660A006F6E0042656C6C3A84
:1003F000204F6E0A0059454C4C4F57004C696768B6
:10040000743A2059656C6C6F770A004C69676874A0
:100410003A205265640A00464C4153485245440014
:100420004C696768743A20466C6173682052656451
:100430000A00646F776E00476174653A20446F77F5
:100440006E0A00475245454E005369676E616C3A2B
:1004500020477265656E0A0054696D656F7574207A
:10046000696E2000730A0054696D652072657365BA
:100470007420627920747261696E0A0054696D6536
:1004800064206F75740A005369676E616C3A20527C
:1004900065640A0042656C6C3A204F66660A004744
:1004A0006174653A2055700A004C696768743A2097
:0504B0004F66660A0022
:00000001FF
